:0200000480007A
:100000006F00C004732F2034930F8000630AFF0336
:10001000930F90006306FF03930FB0006302FF038A
:10002000170F0080130F0FFE63040F0067000F000F
:10003000732F203463540F006F004000136E9E53E3
:10004000171F00002320CFFD6FF09FFF732540F1A5
:100050006310050073251030635805000F00F00F82
:10006000130E100073000000130E00009702000032
:10007000938282F973905230735020307350303035
:1000800073504030970200809382C2F7638C020065
:10009000739052109302B01A739022307323203061
:1000A000E39E62F873500030970200009382420191
:1000B00073901234732540F17300203093000000D8
:1000C00013010000B3912002930E0000130E2000D4
:1000D000639AD14B9300100013011000B3912002DA
:1000E000930E0000130E3000639ED1499300300040
:1000F00013017000B3912002930E0000130E400014
:100100006392D149930000003781FFFFB391200231
:10011000930E0000130E50006396D147B700008085
:1001200013010000B3912002930E0000130E600033
:10013000639AD145B700008013010000B3912002FB
:10014000930E0000130E7000639ED143B7B0AAAAAD
:100150009380B0AA370103001301D1E7B3912002C5
:10016000B70EFFFF938E1E08130EE001639CD14172
:10017000B70003009380D0E737B1AAAA1301B1AA50
:10018000B3912002B70EFFFF938E1E08130EF001ED
:10019000639AD13FB70000FF370100FFB3912002FF
:1001A000B70E0100130E0002639ED13D9300F0FFD5
:1001B0001301F0FFB3912002930E0000130E100202
:1001C0006392D13D9300F0FF13011000B391200220
:1001D000930EF0FF130E20026396D13B93001000A4
:1001E0001301F0FFB3912002930EF0FF130E3002C3
:1001F000639AD139B700D0003701B000B390200224
:10020000B79E0000938E0EF0130E8000639CD037D3
:10021000B700E0003701B00033912002B7AE000014
:10022000938E0EA0130E9000631ED135B700D00040
:10023000B3901002B7BE0000938E0E90130EA00074
:100240006392D03513020000B700D0003701B00030
:10025000B3912002138301001302120093022000C5
:10026000E31452FEB79E0000938E0EF0130EB00002
:10027000631AD33113020000B700E0003701B00069
:10028000B391200213000000138301001302120037
:1002900093022000E31252FEB7AE0000938E0EA030
:1002A000130EC0006310D32F13020000B700F0003C
:1002B0003701B000B39120021300000013000000CA
:1002C000138301001302120093022000E31052FE78
:1002D000B7AE0000938E0E50130ED0006314D32BD4
:1002E00013020000B700D0003701B000B391200224
:1002F0001302120093022000E31652FEB79E000084
:10030000938E0EF0130EE000639ED12713020000BF
:10031000B700E0003701B00013000000B3912002E5
:100320001302120093022000E31452FEB7AE000045
:10033000938E0EA0130EF0006396D12513020000D9
:10034000B700F0003701B0001300000013000000F8
:10035000B39120021302120093022000E31252FE16
:10036000B7AE0000938E0E50130E0001639CD12196
:1003700013020000B700D000130000003701B000E6
:10038000B39120021302120093022000E31452FEE4
:10039000B79E0000938E0EF0130E10016394D11FD0
:1003A00013020000B700E000130000003701B000A6
:1003B00013000000B39120021302120093022000E8
:1003C000E31252FEB7AE0000938E0EA0130E200172
:1003D000639AD11B13020000B700F0001300000065
:1003E000130000003701B000B39120021302120085
:1003F00093022000E31252FEB7AE0000938E0E501F
:10040000130E30016390D119130200003701B000C0
:10041000B700D000B3912002130212009302200013
:10042000E31652FEB79E0000938E0EF0130E4001AD
:10043000639AD115130200003701B000B700E00045
:1004400013000000B3912002130212009302200057
:10045000E31452FEB7AE0000938E0EA0130E5001AF
:100460006392D113130200003701B000B700F0000F
:100470001300000013000000B391200213021200C9
:1004800093022000E31252FEB7AE0000938E0E508E
:10049000130E60016398D10F130200003701B00002
:1004A00013000000B700D000B39120021302120025
:1004B00093022000E31452FEB79E0000938E0EF0CC
:1004C000130E70016390D10D130200003701B000CC
:1004D00013000000B700E00013000000B3912002F9
:1004E0001302120093022000E31252FEB7AE000086
:1004F000938E0EA0130E80016396D10913020000A3
:100500003701B0001300000013000000B700F00036
:10051000B39120021302120093022000E31252FE54
:10052000B7AE0000938E0E50130E9001639CD10560
:10053000B700007C33111002930E0000130EA001CF
:100540006312D105B700008033910002930E0000C2
:10055000130EB0016318D103B3100002930E000014
:10056000130EC0016390D003B700100237012002C0
:1005700033902002930E0000130ED0016314D001BB
:10058000631CC0010F00F00F63000E00131E1E005D
:10059000136E1E00730000000F00F00F130E10000A
:1005A00073000000731000C0000000000000000095
:1005B000000000000000000000000000000000003B
:0405C0000000000037
:1010000000000000000000000000000000000000E0
:1010100000000000000000000000000000000000D0
:1010200000000000000000000000000000000000C0
:1010300000000000000000000000000000000000B0
:081040000000000000000000A8
:040000058000200057
:00000001FF
